:0200000480007A
:10000000B72F0000938F0F8073900F3015A8130047
:100010000000130000001300000013000000130094
:100020000000130000001300000013000000130084
:100030000000130000001300000013000000010086
:10004000970200009382020C73905230814001416C
:100050008141014281420143814301448144014580
:100060008145014681460147814701488148014950
:100070008149014A814A014B814B014C814C014D20
:10008000814D014E814E014F814F971102009381A6
:1000900021B6170502001305E536979503009385F1
:1000A000256801461122170502001305A53397059F
:1000B00002009385A5330146C52817A50300130543
:1000C000656697B503009385A56537B6ABAB130698
:1000D000B6BAD92817B103001301C164EF40D01E8E
:1000E000860293D21200F512638802008242110147
:1000F0006F00001073002030824211017300203025
:10010000711116C0F3222034E3CC02FC82421101AB
:10011000130141F806C20AC40EC612C816CA1ACC88
:100120001ECE22D026D22AD42ED632D836DA3ADCC7
:100130003EDEC2C0C6C2CAC4CEC6D2C8D6CADACC97
:10014000DECEE2D0E6D2EAD4EED6F2D8F6DAFADCA7
:10015000FEDE73252034F32510340A8601A07310C7
:10016000153492402241B2414242D2426243F243AC
:10017000025492542255B2554256D2566257F25703
:10018000064896482649B649464AD64A664BF64B33
:10019000065C965C265DB65D465ED65E665FF65F83
:1001A0001301C1077300203010C16374B50011053D
:1001B000E5BF828000000000000000000000000099
:1001C000000000000000000000000000000000002F
:1001D000000000000000000000000000000000001F
:1001E000000000000000000000000000000000000F
:1001F000197106C00AC20EC412C616C81ACA1ECC8D
:1002000022CE26D02AD22ED432D636D83ADA3EDCC6
:1002100042DEC6C0CAC2CEC4D2C6D6C8DACADECC96
:10022000E2CEE6D0EAD2EED4F2D6F6D8FADAFEDCA6
:100230009702020083A2021B23A02200F3221034A3
:1002400096DEEF006030170102000321A119024180
:10025000F65273901234B72200009382028873A082
:10026000023082403242C2425243E24372448254DC
:100270001255A2553256C2565257E2577258864806
:100280001649A649364AC64A564BE64B764C865C1A
:10029000165DA65D365EC65E565FE65F0961730059
:1002A0002030970202009382E21523A0120023A2BD
:1002B000220023A4320023A6420023A8520023AA2E
:1002C000620023AC720023AE820023A0920223A21C
:1002D000A20223A4B20223A6C20223A8D20223AA06
:1002E000E20223ACF20223AE020323A0120523A2F2
:1002F000220523A4320523A6420523A8520523AADA
:10030000620523AC720523AE820523A0920723A2C7
:10031000A20723A4B20723A6C20723A8D20723AAB1
:10032000E20723ACF207EF40E06E17010200032161
:10033000610B0241F65273901234B722000093828F
:10034000028873A0023082403242C2425243E243EA
:10035000724482541255A2553256C2565257E25731
:10036000725886481649A649364AC64A564BE64B45
:10037000764C865C165DA65D365EC65E565FE65FB1
:10038000096173002030970202009382A20783A0C4
:10039000020003A1420083A1820003A2C20083A243
:1003A000020103A3420183A3820103A4C20183A427
:1003B000020203A5420283A5820203A6C20283A60B
:1003C000020303A7420383A7820303A8C20383A8EF
:1003D000020403A9420483A9820403AAC20483AAD3
:1003E000020503AB420583AB820503ACC20583ACB7
:1003F000020603AD420683AD820603AEC20683AE9B
:10040000020703AFC20983AF820782807370043092
:10041000197106C00AC20EC412C616C81ACA1ECC6A
:1004200022CE26D02AD22ED432D636D83ADA3EDCA4
:1004300042DEC6C0CAC2CEC4D2C6D6C8DACADECC74
:10044000E2CEE6D0EAD2EED4F2D6F6D8FADAFEDC84
:100450009702020083A202F923A0220086DEEF1099
:100460003062170102000321E1F70241F652739056
:100470001234B72200009382028873A002308240B7
:100480003242C2425243E243724482541255A25550
:100490003256C2565257E257725886481649A649F4
:1004A000364AC64A564BE64B764C865C165DA65DD0
:1004B000365EC65E565FE65F0961730020309707BF
:1004C00002009387E7F29843FD576305F7007370C6
:1004D000043001A07370043001A041112AC6B24754
:1004E000739047300100410182804111F327403071
:1004F0003EC673F04330B2473E85410182804111D0
:100500002AC62EC432C2B247F1173EC62247B247AE
:1005100098C3B247938787FA3EC61247B24798C33B
:10052000B247A1173EC68E873E87B24798C3B247EF
:10053000D1173EC6170700001307A7F8B24798C3A4
:10054000B2473E8541018280411106C6EF402045F9
:10055000EF105036AA8799C3EF1090520100B240B5
:100560004101828041112AC6B24713878700B247F2
:10057000D8C3B2477D5798C7B24713878700B247A1
:10058000D8C7B24713878700B24798CBB24723A09A
:10059000070001004101828041112AC6B24723A809
:1005A000070001004101828001112AC62EC4B24712
:1005B000DC433ECEA2477247D8C3F2479847A247D2
:1005C00098C7F2479C472247D8C3F247224798C7AB
:1005D000A247324798CBB2479C4313871700B247D4
:1005E00098C301000561828001112AC62EC4A2476A
:1005F0009C433ECC6247FD576316F700B2479C4BC5
:100600003ECE31A8B247A1073ECE21A0F247DC433F
:100610003ECEF247DC439C436247E379F7FEF24764
:10062000D843A247D8C3A247DC43224798C7A24772
:10063000724798C7F2472247D8C3A247324798CBA0
:10064000B2479C4313871700B24798C30100056166
:10065000828001112AC6B2479C4B3ECEB247DC4392
:100660003247184798C7B2479C4732475843D8C3C8
:10067000F247DC4332476316F700B2479847F24728
:10068000D8C3B24723A80700F2479C431387F7FF5C
:10069000F24798C3F2479C433E8505618280797199
:1006A00006D622D42AC62EC4B2473ECEF24781E7F0
:1006B0007370043001A0EF20A078F2478043F24726
:1006C000D85FF247BC43BE853A85EF50E065AA8704
:1006D0003307F400F247D8C3F24723AC0702F247CE
:1006E0009843F24798C7F2478043F247DC5F13878D
:1006F000F7FFF247BC43BE853A85EF50E062AA8718
:100700003307F400F247D8C7F2477D57F8C3F247E2
:100710007D57B8C7A24799EFF2479C4B8DC7F24768
:10072000C1073E85EF1010622A878547631DF700D9
:10073000F13911A8F247C1073E852D35F24793875D
:1007400047023E850535EF20807285473E85B250D1
:10075000225445618280797106D62AC62EC4B2879A
:10076000A303F10002CCB24781E77370043001A00B
:10077000A24799E302CE01A8A2453245EF50C05AE4
:10078000AA8785073ECEF247938747053E85EF301F
:10079000007E2ACAD24785CFA24789E7D24752476F
:1007A00098C331A0D24713874705D24798C3D24791
:1007B0003247D8DFD2472247B8C385455245C535B1
:1007C000D247034771002388E704D2473ECCE24773
:1007D00081E77370043001A0E2473E85B250456165
:1007E0008280797106D6AA87A307F1001305400518
:1007F000EF30E0772ACEF247B9CFF24723A20700C5
:10080000F24723A00700F24723A40700F24723A6DC
:100810000700F24723AC0702F2470547D8DFF2474B
:1008200023A00704F2477D57F8C3F2477D57B8C7A6
:10083000F2470347F1002388E704F247C1073E85EA
:100840001533F247938747023E85293B814601468F
:10085000814572453122F2473E85B2504561828022
:10086000797106D622D42AC6B2473ECCE24781E748
:100870007370043001A0E247C043EF20803EAA8796
:100880006313F402E247DC471387F7FFE247D8C758
:10089000E247DC4791E78146014681456245C92030
:1008A00085473ECE11A002CEF2473E85B25022547B
:1008B00045618280797106D622D42AC62EC4B247F9
:1008C0003ECCE24781E77370043001A0E247C043A9
:1008D000EF202039AA87631BF400E247DC47138727
:1008E0001700E247D8C785473ECE0DA08146224675
:1008F00081456245812B2ACE724785476318F700F0
:10090000E247DC4713871700E247D8C7F2473E8526
:10091000B250225445618280797106D62AC62EC40F
:10092000B24781E77370043001A02247B24763F5F4
:10093000E7007370043001A0094681453245213D2E
:100940002ACEF24781C7F247224798DFF24781E774
:100950007370043001A0F2473E85B2504561828039
:10096000397106DE2AC62EC432C236C002D6B2475C
:100970003ED4A25781E77370043001A0A24781E7FB
:10098000A257BC4399E3854711A0814781E7737063
:10099000043001A0024789476317F700A257D85FC8
:1009A00085476314F700854711A0814781E773707D
:1009B000043001A0EF20402CAA8799E3924799E3E5
:1009C000854711A0814781E77370043001A0EF20B3
:1009D0002047A257985FA257DC5F6366F700024783
:1009E0008947631EF7020246A2452255EF00007CAC
:1009F0002AD2A257DC5389CFA257938747023E855C
:100A0000EF1050342A8785476317F700013421A07F
:100A1000925791C3E53AEF20804585474DA0924714
:100A200089E7EF20C044814759A8B25799E77C086D
:100A30003E85EF10D04885473ED6EF204043EF106B
:100A4000A03BEF20E03FA257F843FD576315F700A6
:100A5000A25723A20704A257B847FD576315F70012
:100A6000A25723A40704EF20804058007C08BA85D1
:100A70003E85EF10D047AA878DEF2255EF00D012A8
:100A8000AA8795C3A257C1071247BA853E85EF10C2
:100A900050122255EF00B003EF10C037AA87E39839
:100AA00007F2AD322DB72255EF007002EF108036FD
:100AB00039BF2255EF00B001EF10C03581473E85A8
:100AC000F25021618280797106D62AC62EC432C2C4
:100AD00036C002CEB2473ECCE24781E773700430A5
:100AE00001A0A24781E7E247BC4399E3854711A0F3
:100AF000814781E77370043001A0EF206034E24742
:100B0000985FE247DC5F6379F7020246A2456245DF
:100B1000EF00C069E247DC5381CFE2479387470289
:100B20003E85EF1030222A8785476313F700F93896
:100B3000EF20E033854785A0924789E7EF202033F7
:100B4000814791A8F24799E71C083E85EF1030379E
:100B500085473ECEEF20A031EF20802E58001C08A4
:100B6000BA853E85EF10B038AA8799EF6245EF004D
:100B7000B003AA8791CFE247C1071247BA853E85E5
:100B8000EF103003613029A0EF20602E814721A0B3
:100B9000EF20E02D9DB73E85B250456182803971CE
:100BA00006DE2AC62EC432C236C002D6B2473ED4B2
:100BB000A25781E77370043001A0A24781E7A257D2
:100BC000BC4399E3854711A0814781E773700430E6
:100BD00001A0EF20E026A2579C5FB5CBA257DC47CF
:100BE0003ED2A2452255792D824795EFA2579C5FB0
:100BF0001387F7FFA25798DFA2579C4391E7EF2096
:100C0000602E2A87A257D8C3A2579C4B8DCFA257DC
:100C1000C1073E85EF1010132A8785476315F70239
:100C2000EFF0CFFE0DA0A2571257D8C7A257DC5342
:100C300099CBA257938747023E85EF10B010AA8741
:100C400099C3EFF0AFFCEF2080228547ADA8924713
:100C500089E7EF20C0218147BDA0B25799E77C0802
:100C60003E85EF10D02585473ED6EF204020EF206F
:100C7000201D58007C08BA853E85EF105027AA87B2
:100C800085EF2255E92DAA8785CFA2579C4391EB8A
:100C9000EF20001BA257DC433E85EF20E000EF2051
:100CA000001DA257938747021247BA853E85EF1071
:100CB0004070EFF0AFF529A0EF20601B814721A025
:100CC000EF20E01A39B73E85F250216182807971B8
:100CD00006D62AC62EC432C236C0B2473ECCE24740
:100CE00081E77370043001A0A24781E7E247BC436B
:100CF00099E3854711A0814781E77370043001A013
:100D0000024789476317F700E247D85F85476314B6
:100D1000F700854711A0814781E77370043001A077
:100D2000EFF0AFFCAA873ECAE247985FE247DC5F7C
:100D30006366F700024789476315F7040246A24538
:100D40006245AD21E247B847FD576313F702E2471A
:100D5000DC538DC7E247938747023E85EF10807EC4
:100D6000AA8789CF924799CB9247054798C339A064
:100D7000E247BC4713871700E247B8C785473ECE16
:100D800011A002CED2473E85EFF02FF5F2473E8507
:100D9000B25045618280797106D62AC62EC4B24708
:100DA0003ECCE24781E77370043001A0E247BC43C8
:100DB00081C77370043001A0E2479C4381E7E2479A
:100DC000DC4399E3854711A0814781E773700430C4
:100DD00001A0EFF08FF1AA873ECAE247985FE24791
:100DE000DC5F6377F704E2479C5F13871700E247F5
:100DF00098DFE247B847FD576313F702E247DC5339
:100E00008DC7E247938747023E85EF10A073AA87FC
:100E100089CFA24799CBA247054798C339A0E2479B
:100E2000BC4713871700E247B8C785473ECE11A0DD
:100E300002CED2473E85EFF04FEAF2473E85B250F0
:100E400045618280397106DE2AC62EC432C236C0A0
:100E500002D6B2473ED4A25781E77370043001A096
:100E6000A24781E7A257BC4399E3854711A0814778
:100E700081E77370043001A0EF101060AA8799E336
:100E8000924799E3854711A0814781E77370043049
:100E900001A0EF10F07AA2579C5FB5CBA257DC47B8
:100EA0003ED2A2452255F92E824795EFA2579C5F6C
:100EB0001387F7FFA25798DFA2579C4391E7EF20D3
:100EC00060022A87A257D8C3A2579C4B8DCFA25746
:100ED000C1073E85EF1000672A8785476315F70233
:100EE000EFF0CFD20DA0A2571257D8C7A257DC53AC
:100EF00099CBA257938747023E85EF10A064AA873B
:100F000099C3EFF0AFD0EF10907685475DA8924778
:100F100089E7EF10D07581476DA0B25799E77C083B
:100F20003E85EF10C07985473ED6EF105074EF0034
:100F3000B06CEF10F070A257F843FD576315F7003F
:100F4000A25723A20704A257B847FD576315F7001D
:100F5000A25723A40704EF10907158007C08BA85AB
:100F60003E85EF10C078AA87A1EB2255CD2EAA8727
:100F70009DCFA2579C4391EBEF10906CA257DC439E
:100F80003E85EF107052EF10906EA2579387470284
:100F90001247BA853E85EF10C04122550D2EEF0055
:100FA0007067AA87E39707EEEFF04FC6DDB52255CD
:100FB000392EEF003066F1BD2255112EEF009065FD
:100FC00081473E85F25021618280797106D62AC61A
:100FD0002EC432C2B2473ECCE24781E77370043080
:100FE00001A0A24781E7E247BC4399E3854711A0EE
:100FF000814781E77370043001A0EFF00FCFAA871B
:101000003ECAE2479C5FA1CBA2456245A52CE247C0
:101010009C5F1387F7FFE24798DFE247F843FD57ED
:101020006312F702E2479C4B85C7E247C1073E8542
:10103000EF104051AA8789CF924799CB9247054735
:1010400098C339A0E247FC4313871700E247F8C36F
:1010500085473ECE11A002CED2473E85EFF0EFC7C6
:10106000F2473E85B25045618280797106D62AC624
:101070002EC4B2473ECCE24781E77370043001A032
:10108000A24781E7E247BC4399E3854711A0814726
:1010900081E77370043001A0E247BC4381E77370BD
:1010A000043001A0EFF06FC4AA873ECAE2479C5FFC
:1010B00089CFE247DC473EC8A2456245E122E247CC
:1010C0004247D8C785473ECE11A002CED2473E85C3
:1010D000EFF0AFC0F2473E85B25045618280797132
:1010E00006D62AC6B24781E77370043001A0EF101C
:1010F0003055B2479C5F3ECEEF107057F2473E85A9
:10110000B25045618280797106D62AC6B2473ECE7A
:10111000F24781E77370043001A0EF107052F2477C
:10112000D85FF2479C5FB307F7403ECCEF103054D6
:10113000E2473E85B2504561828001112AC6B2471E
:1011400081E77370043001A0B2479C5F3ECEF24746
:101150003E8505618280797106D62AC6B2473ECEA9
:10116000F24781E77370043001A07245E5247245AF
:10117000EF20F0720100B2504561828041112AC611
:10118000B247FC473E854101828041112AC62EC4E8
:10119000B2472247F8C701004101828041112AC6A7
:1011A000B24783C707053E8541018280797106D623
:1011B0002AC62EC432C202CEB247BC4391EFB24718
:1011C0009C43D5E7B247DC433E85EF10903B2ACEE7
:1011D000B24723A2070061A8924785EFB24798471C
:1011E000B247BC433E86A2453A85EF20F079B2472C
:1011F0009847B247BC433E97B24798C7B247984713
:10120000B247DC436365F706B2479843B24798C7D5
:10121000B9A8B247D847B247BC433E86A2453A85F3
:10122000EF209076B247D847B247BC43B307F040AF
:101230003E97B247D8C7B247D847B2479C43637B73
:10124000F700B247D843B247BC43B307F0403E97DC
:10125000B247D8C712478947631BF700B2479C5F64
:1012600099C7B2479C5F1387F7FFB24798DFB24731
:101270009C5F13871700B24798DFF2473E85B25054
:1012800045618280011106CE2AC62EC4B247BC43F6
:101290009DCBB247D847B247BC433E97B247D8C769
:1012A000B247D847B247DC436366F700B24798437A
:1012B000B247D8C7B247D847B247BC433E86BA8583
:1012C0002245EF20706C0100F2400561828001111F
:1012D00006CE2AC6EF10D03625A0B247DC5395C7FC
:1012E000B247938747023E85EF10C025AA8799C36E
:1012F000EF104049B247BC471387F7FFB247B8C762
:10130000B247BC47E34BF0FC11A00100B2477D5748
:10131000B8C7EF10D035EF10B0321DA0B2479C4BCC
:101320008DC7B247C1073E85EF10C021AA8799C378
:10133000EF104045B247FC431387F7FFB247F8C3AD
:10134000B247FC43E34CF0FC11A00100B2477D57CB
:10135000F8C3EF10D0310100F2400561828079714D
:1013600006D62AC6EF10D02DB2479C5F81E785478D
:101370003ECE11A002CEEF10902FF2473E85B25024
:101380004561828001112AC6B24781E7737004303B
:1013900001A0B2479C5F81E785473ECE11A002CEF7
:1013A000F2473E8505618280797106D62AC6EF1024
:1013B0003029B247985FB247DC5F6315F700854775
:1013C0003ECE11A002CEEF10902AF2473E85B250D9
:1013D0004561828001112AC6B24781E773700430EB
:1013E00001A0B247985FB247DC5F6315F7008547FD
:1013F0003ECE11A002CEF2473E85056182800111EA
:101400002AC62EC402CE81A0178703001307872D9A
:10141000F2478E07BA979C4385E7178703001307A7
:10142000672CF2478E07BA97224798C317870300A5
:101430001307472BF2478E07BA973247D8C301A844
:10144000F24785073ECE72479D47E3FFE7FA01006A
:101450000561828001112AC602CE0DA817870300FC
:1014600013074728F2478E07BA97DC433247631CBD
:10147000F700178703001307E726F2478E07BA978E
:1014800023A0070001A8F24785073ECE72479D477B
:10149000E3F6E7FC010005618280797106D62AC671
:1014A0002EC432C2B2473ECEEF109019F247F84335
:1014B000FD576315F700F24723A20704F247B84728
:1014C000FD576315F700F24723A40704EF10301A05
:1014D000F2479C5F89EBF247938747021246A24589
:1014E0003E85EF00907E7245DD330100B2504561CC
:1014F0008280397106DE2ACE2ECC36C83AC63EC46A
:1015000042C246C0B287231BF100F24781E77370E5
:10151000043001A03247A54763F5E700737004303B
:1015200001A08357610192453E85EF1080512AD476
:10153000A257638F0712A257985B83566101B707C2
:101540000040FD17B6978A07BA973ED29257F19B93
:101550003ED292578D8B81C77370043001A08357A0
:1015600061013E8782463246E2452255EF10E02770
:101570004246F2451255EFE09FF82A87A25798C3DA
:10158000A24781C7A247225798C3EF10700B97F765
:101590000100938767029C431387170097F70100A8
:1015A0009387870198C397F701009387A7E39C432C
:1015B00095E397F701009387E7E2225798C397F7DF
:1015C0000100938767FF98438547631AF702EF107E
:1015D000C02C35A097F701009387C7FE9C4385E395
:1015E00097F70100938707E09C43DC573247636815
:1015F000F70097F701009387E7DE225798C397F724
:101600000100938727FD9C431387170097F701007C
:10161000938747FC98C397F701009387A7FB9843EC
:10162000A257B8C7A257D85797F70100938747F931
:101630009C4363F9E700A257D85797F701009387B7
:1016400027F898C3A257D857BA878A07BA978A0744
:1016500017F701001307C7E23E97A2579107BE850F
:101660003A85EFE07FF485473ED6EF10500019A091
:10167000FD573ED6325785476313F70297F70100AF
:10168000938747F49C4381CF97F70100938787D5D1
:101690009C43DC57324763F4E700EFE03FD7B25793
:1016A0003E85F25021618280797106D62AC6EF10FC
:1016B0002079B24799E797F701009387A7D29C4317
:1016C00011A0B2473ECEF24791073E85EFE07FF88A
:1016D000F2479C5791C7F247E1073E85EFE07FF75D
:1016E000F2479107BE8517F50100130525EAEFE0E3
:1016F000BFEB97F701009387A7EA9C431387170076
:1017000097F701009387C7E998C397F7010093877C
:1017100067EC9C431387170097F70100938787EBCB
:1017200098C3EF10C07497F701009387A7E99C4313
:101730009DCB97F701009387E7CA9C437247631ECE
:10174000F70097F70100938767E99C4381C773709F
:10175000043001A0EFE09FCB39A0EF10606EEF10D6
:10176000A04BEF10C0700100B250456182807971CA
:1017700006D62AC62EC402CEB24781E77370043063
:1017800001A0A24781E77370043001A097F7010020
:101790009387C7E49C4381C77370043001A0A92DCF
:1017A00097F70100938787E19C433ECCB2479C4367
:1017B0002247BA973ECAB2479C436247637EF7000E
:1017C000B2479C4352476374F7025247E24763F0C3
:1017D000E70285473ECE21A8B2479C435247636645
:1017E000F7005247E24763F4E70085473ECEB24731
:1017F000524798C3F24789CF97F70100938787BE76
:101800009C4391073E85EFE0DFE45245EF10001B5B
:1018100011252AC8C24799E3EFE05FBF0100B2502B
:1018200045618280797106D62AC602CEB247A9C325
:1018300097F70100938787DA9C4381C77370043060
:1018400001A05D2B97F70100938747D79C43324750
:10185000BA973ECC97F701009387C7B89C4391078E
:101860003E85EFE01FDF6245EF10401565232ACE6D
:10187000F24799E3EFE09FB90100B25045618280E1
:10188000797106D62AC6B2473ECCE24781E773702B
:10189000043001A097F701009387C7B49C436247C7
:1018A0006314F70002CEBDA0EF108059E247DC4B75
:1018B0003ECAEF10C05B97F70100938767CB9C434C
:1018C0005247630AF70097F701009387A7CA9C4322
:1018D00052476315F70089473ECE2DA8524797F728
:1018E0000100938727CC631BF700E2479C5781E7F1
:1018F0008D473ECE05A089473ECE29A8524797F78F
:1019000001009387A7C86315F70091473ECE19A041
:1019100085473ECEF2473E85B2504561828079715F
:1019200006D62AC6EF10C051B24799E797F70100D3
:10193000938747AB9C4311A0B2473ECEF247DC579A
:101940003ECCEF10C052E2473E85B25045618280E6
:10195000797106D62AC6EFE05FB9AA873ECEB247B4
:1019600099E797F701009387E7A79C4311A0B24737
:101970003ECCE247DC573ECAF2473E85EFE0FFB57A
:10198000D2473E85B25045618280797106D62AC61B
:101990002EC402CE2247A54763F5E70073700430DA
:1019A00001A02247A54763F4E700A5473EC4EF1016
:1019B0002049B24799E797F701009387A7A29C4374
:1019C00011A0B2473ECCE247BC4B3ECA5247A247A9
:1019D000630AF70E2247D24763F6E70297F7010042
:1019E000938747A09C4362476308F70297F701007B
:1019F0009387479F9C43DC572247636FF7008547D7
:101A00003ECE19A897F701009387C79D9C43624774
:101A10006314F70085473ECEE247DC573EC8E247F5
:101A2000B84BE247DC576315F700E2472247D8D7A7
:101A3000E2472247B8CBE2479C4F63C707002947DC
:101A4000A2471D8FE24798CFE247D44B4247BA875F
:101A50008A07BA978A0717F70100130767A2BA9790
:101A60006394F600854711A08147B9C7E247910703
:101A70003E85EFE01FBEE247D85797F701009387F6
:101A800027B49C4363F9E700E247D85797F7010072
:101A9000938707B398C3E247D857BA878A07BA979C
:101AA0008A0717F701001307A79D3E97E2479107A2
:101AB000BE853A85EFE05FAF724785476314F70054
:101AC000EFE0DF94EF10A03A0100B2504561828050
:101AD000797106D62AC6EF10A036B24799E797F774
:101AE0000100938727909C4311A0B2473ECEF24756
:101AF00091073E85EFE0FFB5F2479C5791C7F2474B
:101B0000E1073E85EFE0FFB4F2479107BE8517F588
:101B10000100130525A9EFE03FA9EF10403597F725
:101B200001009387278C9C4372476319F70497F74A
:101B30000100938727A99C4389CF97F701009387DA
:101B4000E7A99C4381C77370043001A0EFE01F8CAC
:101B500091A097F701009387E7A4984397F70100B6
:101B6000938787A59C436319F70097F70100938734
:101B7000678723A0070039A8212729A897F7010024
:101B8000938747A49C4399C7EF10802BEF10C008A0
:101B9000EF10E02D0100B2504561828001112AC68C
:101BA00002CEB2473ECCB24781E77370043001A049
:101BB000E247D84B97F701009387C79E6314F7005D
:101BC000854711A0814795C3E247985797F70100D1
:101BD0009387879A630BF700E2479C5799E3854701
:101BE00011A0814799C385473ECEF2473E850561E6
:101BF0008280797106D62AC6B2473ECEB24781E7C7
:101C00007370043001A0F247C9C797E701009387BA
:101C1000677D9C437247630EF706EF1060227245A2
:101C2000B53F2A8785476314F706F24791073E853B
:101C3000EFE03FA2F247D85797F701009387479804
:101C40009C4363F9E700F247D85797F70100938761
:101C5000279798C3F247D857BA878A07BA978A074F
:101C600017F701001307C7813E97F2479107BE851A
:101C70003A85EFE07F93F247D85797E701009387C3
:101C800067769C43DC576364F700EFE02FF8EF10B2
:101C9000001E0100B25045618280797106D62AC6C5
:101CA00002CEB2473ECCB24781E77370043001A048
:101CB000EFE0BF83AA873ECA6245CD352A878547B4
:101CC0006314F70897F70100938747919C43A5E7B2
:101CD000E247D85797E701009387C7709C43DC57CA
:101CE0006364F70085473ECEE24791073E85EFE00B
:101CF0005F96E247D85797F701009387678C9C431C
:101D000063F9E700E247D85797F701009387478BBD
:101D100098C3E247D857BA878A07BA978A0717E75E
:101D200001001307E7753E97E2479107BE853A85A4
:101D3000EFE09F8711A8E247E107BE8517F5010094
:101D400013058583EFE05F86D2473E85EFE0EFF82D
:101D5000F2473E85B25045618280011106CE81482E
:101D600001488147014781461306004097E501007D
:101D70009385452917150000130585A5EFF06FF72A
:101D80002AC6324785476315F700EF10C06D2AC693
:101D9000324785476319F7027370043097F70100E3
:101DA000938787837D5798C397F70100938787812F
:101DB000054798C397F701009387478023A0070042
:101DC000EFE02FCE31A0B24781E77370043001A05D
:101DD0000100F24005618280411106C67370043033
:101DE00097E701009387077E23A00700EFE0AFD9B4
:101DF0000100B2404101828097E701009387077E8E
:101E00009C431387170097E701009387277D98C3AA
:101E100001008280011106CE02C697E70100938778
:101E2000E77B9C4381E77370043001A0EF10400111
:101E300097E701009387877A9C431387F7FF97E71B
:101E400001009387A77998C397E7010093870779E3
:101E50009C436390071097E701009387E7759C43C5
:101E60006389070E59A097E701009387E770DC4765
:101E7000DC473EC4A247E1073E85EFE08FFDA24765
:101E800091073E85EFE0EFFCA247D85797E70100A6
:101E9000938707739C4363F9E700A247D85797E7F6
:101EA00001009387E77198C3A247D857BA878A077A
:101EB000BA978A0717E701001307875C3E97A24786
:101EC0009107BE853A85EFE02FEEA247D85797E7F6
:101ED0000100938727519C43DC576368F70097E71D
:101EE00001009387A76E054798C397E70100938782
:101EF000A7689C43ADFB97E701009387E76C9C4381
:101F00008DCF35A0452AAA8799C797E70100938707
:101F1000E76B054798C397E701009387E76A9C43FF
:101F20001387F7FF97E701009387076A98C397E73E
:101F30000100938767699C43F1F797E70100938756
:101F4000E768984385476316F70085473EC6EFE08C
:101F5000EFCBEF00D071B2473E85F2400561828041
:101F6000011106CEEF00D06D97E70100938707655A
:101F70009C433EC6EF00B06FB2473E85F24005611C
:101F80008280011106CEEFE04FD6AA873EC697E7C2
:101F900001009387A7629C433EC4B2473E85EFE0B1
:101FA000CFD3A2473E85F2400561828097E70100CA
:101FB000938787609C433E858280797106D62AC6C6
:101FC0002EC432C202CEA9473ECC3D3597E7010070
:101FD0009387875E9C4322476368F70CE247FD17AF
:101FE0003ECCF24796073247B306F7006247BA87FE
:101FF0008A07BA978A0717E7010013076748BA9755
:102000000546BE853685EF00902A2A87F247BA97A3
:102010003ECEE247E1F7F247960732473E9797E711
:1020200001009387E7549C430946BE853A85EF003B
:1020300010282A87F247BA973ECEF24796073247D2
:102040003E9797E701009387E7529C430946BE8578
:102050003A85EF00D0252A87F247BA973ECEF2475D
:1020600096073247BA97114697E5010093850552C6
:102070003E85EF00D0232A87F247BA973ECEF2473B
:1020800096073247BA970D4697E50100938585512B
:102090003E85EF00D0212A87F247BA973ECE92477D
:1020A00081C7924723A00700B533F2473E85B2505F
:1020B00045618280797106D602CE97E70100938749
:1020C000E7519C436395071897E701009387074FF3
:1020D0009C431387170097E701009387274E98C307
:1020E00097E701009387874D9C433ECCE247B9EFC9
:1020F00097E701009387C7479C439C4381C7737050
:10210000043001A097E70100938787469C433ECAAD
:1021100097E7010093870746984397E70100938765
:10212000274598C397E701009387C744524798C350
:1021300097E701009387C7499C431387170097E7E8
:1021400001009387E74898C3EF00102D97E701003F
:10215000938787489C4362476365F70C97E70100C4
:10216000938707419C439C4399E3854711A081478E
:1021700081CB97E70100938727467D5798C355A0E9
:1021800097E701009387C73E9C43DC47DC473EC886
:10219000C247DC433EC66247B2476379F70097E720
:1021A000010093876743324798C3A5A8C2479107A8
:1021B0003E85EFE00FCAC2479C5791C7C247E1076F
:1021C0003E85EFE00FC9C247D85797E701009387D4
:1021D000273F9C4363F9E700C247D85797E70100C0
:1021E0009387073E98C3C247D857BA878A07BA97DA
:1021F0008A0717E701001307A7283E97C2479107F0
:10220000BE853A85EFE04FBAC247D85797E701003D
:102210009387471D9C43DC57E362F7F485473ECE26
:1022200035BF97E701009387E71B9C43D85797E694
:1022300001009386E624BA878A07BA978A07B69779
:102240009843854763F1E70285473ECE29A897E783
:102250000100938767379C431387170097E70100B6
:102260009387873698C397E70100938727369C4367
:1022700099C385473ECEF2473E85B2504561828084
:10228000011106CE97E70100938747359C4381CB28
:1022900097E7010093878733054798C339A297E7EB
:1022A00001009387A73223A0070097E701009387D7
:1022B00067139C439C5B3EC6B7A7A5A59387575A57
:1022C0003EC4B2479C4322476314F702B2479107CA
:1022D0009C432247631EF700B247A1079C43224755
:1022E0006318F700B247B1079C4322476308F7041D
:1022F00097E701009387070F984397E701009387BB
:10230000670E9C4393874703BE853A85EF20100BE9
:1023100035A097E701009387A72A9C4381E7737054
:10232000043001A097E70100938787299C43138716
:10233000F7FF97E701009387A72898C397E7010065
:1023400093870728984397E6010093866613BA8718
:102350008A07BA978A07B6979C43C5DF97E70100BB
:10236000938707269843BA878A07BA978A0717E799
:1023700001001307E710BA973EC29247DC43D843E7
:102380009247D8C39247D8439247A1076317F700F3
:102390009247DC43D8439247D8C39247DC43D8479F
:1023A00097E701009387070498C30100F240056195
:1023B0008280797106D62AC62EC4B24781E773702F
:1023C000043001A097E701009387C7019C43E10710
:1023D000BE853245EFE04FA197E701009387870064
:1023E0009C4391073E85EFE0CFA62247FD5763103F
:1023F000F70297E701009387E7FE9C439107BE85AC
:1024000017E501001305051AEFE00F9A19A897E7E1
:1024100001009387A71A9C432247BA973ECE724584
:10242000712B0100B25045618280797106D62AC6AF
:102430002EC432C2B24781E77370043001A097E71F
:1024400001009387A7199C4381E77370043001A0B2
:1024500097E70100938707F99C43A246370700805E
:10246000558F98CF97E701009387C7F79C43E10703
:10247000BE853245EFE04F9397E70100938787F6DB
:102480009C4391073E85EFE0CF9C1247FD576310B8
:10249000F70297E701009387E7F49C439107BE8515
:1024A00017E5010013050510EFE00F9019A897E755
:1024B00001009387A7109C431247BA973ECE7245FE
:1024C000F5290100B25045618280797106D62AC68D
:1024D0002EC432C2B24781E77370043001A097E77F
:1024E0000100938727F09C43E107BE853245EFE06A
:1024F000AF8B97E701009387E7EE9C4391073E85FA
:10250000EFE02F95124785476310F70297E7010028
:10251000938747ED9C439107BE8517E5010013059E
:102520006508EFE06F8819A897E70100938707090E
:102530009C432247BA973ECE724549210100B250D2
:1025400045618280797106D62AC6B247DC47DC47EE
:102550003ECCE24781E77370043001A0E247E10717
:102560003E85EFE00F8F97E70100938727079C4395
:10257000A1EBE24791073E85EFE0AF8DE247D857E8
:1025800097E701009387C7039C4363F9E700E2479D
:10259000D85797E701009387A70298C3E247D85717
:1025A000BA878A07BA978A0717E70100130747ED2A
:1025B0003E97E2479107BE853A85EFD0FFFE11A80E
:1025C000E247E107BE8517E501001305E5FAEFD004
:1025D000BFFDE247D85797E701009387A7E09C43E8
:1025E000DC5763FBE70085473ECE97E70100938702
:1025F000E7FD054798C311A002CEF2473E85B250D1
:1026000045618280797106D62AC62EC497E70100FB
:102610009387C7FC9C4381E77370043001A0224775
:10262000B70700805D8FB24798C3B247DC473ECC06
:10263000E24781E77370043001A03245EFE06F811B
:10264000E24791073E85EFE0CF80E247D85797E712
:1026500001009387E7F69C4363F9E700E247D85708
:1026600097E701009387C7F598C3E247D857BA8721
:102670008A07BA978A0717E70100130767E03E97B2
:10268000E2479107BE853A85EFD01FF2E247D8575F
:1026900097E70100938707D59C43DC5763FBE7006E
:1026A00085473ECE97E70100938747F2054798C3D9
:1026B00011A002CEF2473E85B250456182804111A1
:1026C0002AC6B24781E77370043001A097E7010082
:1026D000938707F09843B24798C397E70100938721
:1026E000E7ED9843B247D8C3010041018280797178
:1026F00006D62AC62EC4B24781E77370043001A003
:10270000A24781E77370043001A01D2F97E70100F5
:102710009387C7EA9C433ECCA2479843FD57631476
:10272000F70002CE91A8B247984397E7010093873C
:1027300027EA9C43630AF700B247DC4362476365BC
:10274000F70085473ECE0DA8B247DC4362471D8F98
:10275000A2479C436370F702A2479843B247D44311
:10276000E247B387F6403E97A24798C33245813F80
:1027700002CE19A085473ECEDD2DF2473E85B250F0
:102780004561828097E70100938747E4054798C336
:102790000100828001112AC6B24799C7B2473ECCD8
:1027A000E247FC473ECE11A002CEF2473E850561CE
:1027B000828001112AC62EC4B24791C7B2473ECECD
:1027C000F2472247F8C7010005618280011106CE59
:1027D0002AC6852297E70100938787CA98438547D1
:1027E000E3F9E7FEEFD09FC2EDB7397106DE2ACEDE
:1027F0002ECC32CA36C8BA872317F10002D625A0DC
:102800006247B257BA9703C70700F246B257B69766
:10281000238AE7026247B257BA9783C7070089CB7A
:10282000B25785073ED63257BD47E3FBE7FC11A000
:102830000100F247A38107045247A54763F4E7006C
:10284000A5473ECAF2475247D8D7F2475247B8CBBE
:10285000F24723AA0704F24791073E85EFD0DFD362
:10286000F247E1073E85EFD03FD3F247724798CB5E
:102870002947D2471D8FF24798CFF2477247D8D3E6
:10288000F24723A20704F24723AC0704F24723AE22
:1028900007040100F25021618280011106CE02C6B8
:1028A0000DA03247BA878A07BA978A0717E701004F
:1028B000130707BDBA973E85EFD0DFCAB247850739
:1028C0003EC63247A547E3FEE7FC17E501001305C6
:1028D000A5C7EFD03FC917E50100130525C8EFD004
:1028E0007FC817E50100130525C9EFD0BFC717E55D
:1028F00001001305A5C9EFD0FFC617E501001305B8
:1029000065CAEFD03FC697E70100938767C617E710
:102910000100130767C398C397E70100938787C532
:1029200017E70100130787C398C30100F240056150
:102930008280011106CE8DA8EFF00FCC97E7010041
:102940009387C7C49C4393B7170093F7F70F3EC60E
:10295000EFF04FCCB247A9EBE52197E70100938751
:10296000E7C2DC47DC473EC4A24791073E85EFD073
:102970005FCE97E70100938727C49C431387F7FF37
:1029800097E70100938747C398C397E701009387B0
:1029900027C19C431387F7FF97E70100938747C040
:1029A00098C3F1212245912C97E70100938747BFF7
:1029B0009C43D9F30100F24005618280011106CEEB
:1029C0002AC697E701009387E7A19C433247D8C303
:1029D00097E70100938787BE9C4332476372F702F3
:1029E00097E70100938707B9984397E7010093871A
:1029F000679F9C439107BE853A85EFD0FFBE35A8FF
:102A000097E701009387C7B6984397E7010093873C
:102A1000679D9C439107BE853A85EFD0FFBC97E741
:102A20000100938767BB9C4332476378F70097E7C1
:102A30000100938767BA324798C30100F2400561ED
:102A40008280797106D6AA872EC42317F100A24787
:102A500089EB8357E1008A073E85EF104051AA8732
:102A600011A0A2473ECCE24785C313050006EF1034
:102A700000502ACEF24789C7F247624798DB31A05F
:102A80006245EF10C06111A002CEF24781CFF2473C
:102A9000985B8357E1008A073E869305500A3A8582
:102AA000EF104075F2473E85B25045618280397122
:102AB00006DE22DC2AC62EC432C202D6A2479C43BE
:102AC000638D070EA2473ED4A257DC43D843A257DA
:102AD000D8C3A257D843A257A1076317F700A2573C
:102AE000DC43D843A257D8C3A257DC43DC473ED2CD
:102AF000A2473ED08257DC43D8438257D8C382577F
:102B0000D8438257A1076317F7008257DC43D843A5
:102B10008257D8C38257DC43DC473ECEB257960774
:102B20003247BA97724798C3B25796073247BA9757
:102B3000724713074703D8C3B25796073247BA976D
:102B40007247384798C7B25796073247BA97124725
:102B5000D8C7B25796073247BA977247585798CB9B
:102B600012478D47631BF700F2479C5799C7B2572E
:102B700096073247BA970947D8C7B25796073247E0
:102B8000BA977247384BD8CBB25796073247BA97A5
:102B900023AC0700F247945BB257960732473304E1
:102BA000F70036850D20AA87231EF400B25785074B
:102BB0003ED672479257E31DF7F2B2573E85F25068
:102BC00062542161828001112AC602CE39A0B24727
:102BD00085073EC6F24785073ECEB24703C70700CA
:102BE0009307500AE305F7FEF24789833ECEF2478A
:102BF000C207C1833E8505618280011106CE2AC6C7
:102C0000B2479C5B3E85EF1080493245EF1020496A
:102C10000100F24005618280411197E7010093872E
:102C200027959C439C4399E3854711A0814781CB1D
:102C300097E701009387479A7D5798C305A097E7C8
:102C400001009387E7929C43DC47DC473EC6B247CE
:102C5000D84397E701009387279898C30100410163
:102C60008280411197D701009387C7779C433EC666
:102C7000B2473E8541018280411197E70100938769
:102C800067949C4381E785473EC619A897E70100F2
:102C90009387C7949C4381E789473EC611A002C62B
:102CA000B2473E8541018280797106D62AC6B24775
:102CB0003ECEB247F9C3F247D85797D70100938762
:102CC00067729C43DC57637AF70AF2479C4F63CCE8
:102CD000070097D701009387E7709C43DC5729478B
:102CE0001D8FF24798CFF247D44BF247D857BA8797
:102CF0008A07BA978A0717D7010013076778BA9728
:102D00006394F600854711A08147A5C3F247910758
:102D10003E85EFD01F9497D701009387A76C9C4303
:102D2000D857F247D8D7F247D85797E7010093878B
:102D300027899C4363F9E700F247D85797E70100DA
:102D40009387078898C3F247D857BA878A07BA97F4
:102D50008A0717D701001307A7723E97F24791071A
:102D6000BE853A85EFD05F8409A897D70100938785
:102D700067679C43D857F247D8D70100B2504561E6
:102D80008280797106D62AC6B2473ECC02CEB247BF
:102D9000DDC397D701009387E7649C4362476305CF
:102DA000F7007370043001A0E247FC4B81E77370B9
:102DB000043001A0E247FC4B1387F7FFE247F8CB52
:102DC000E247D857E247BC4B6307F706E247FC4BA4
:102DD000BDE3E24791073E85EFD0BF87E247B84B9E
:102DE000E247D8D7E247DC5729471D8FE24798CF03
:102DF000E247D85797D701009387877C9C4363F9B4
:102E0000E700E247D85797D701009387677B98C3BD
:102E1000E247D857BA878A07BA978A0717D70100B7
:102E2000130707663E97E2479107BE853A85EFD0C4
:102E3000AFF785473ECEF2473E85B250456182806E
:102E40007370043097D701009387C7779C4391CF65
:102E500097D70100938707599C43F8430507F8C3A8
:102E600097D70100938707589C430100828097D72A
:102E70000100938727759C438DCB97D701009387DB
:102E800067569C43FC4395C397D7010093878755AA
:102E90009C43F8437D17F8C397D701009387875465
:102EA0009C43FC4399E3736004300100828041112C
:102EB00097D70100938707539C439C4F3EC697D7F3
:102EC0000100938727529C43D85797D701009387D7
:102ED00067519C43A9463387E64098CFB2473E8569
:102EE0004101828097D701009387C74F9C4389CBCC
:102EF00097D701009387074F9C43F84B0507F8CB02
:102F000097D701009387074E9C433E858280797155
:102F100006D62AC62EC42D3797D701009387874C33
:102F20009C43BC4FADE397D701009387A74B9C43CD
:102F30000547F8CFA247A1CB97D701009387874ACF
:102F40009C4391073E85EFD0CFF02247FD57631099
:102F5000F70297D701009387E7489C439107BE8506
:102F600017D5010013050564EFD00FE419A897D712
:102F700001009387A7649C432247BA973ECE7245CF
:102F8000353CEFD0AFC8E535653D97D70100938755
:102F900067459C43BC4F3ECCE2479DC3B24789CBBB
:102FA00097D70100938707449C4323AC070409A8E3
:102FB00097D70100938707439C43B84F7D17B8CF3D
:102FC00097D70100938707429C4323AE07044535FA
:102FD000E2473E85B25045618280797106D62AC6A5
:102FE0002EC432C236C0A93D97D701009387873FD0
:102FF0009C43F84F8947630DF70697D701009387E5
:10300000673E9C43B44F32471347F7FF758FB8CFE5
:1030100097D701009387073D9C430547F8CF824728
:10302000A1CB97D701009387E73B9C4391073E854F
:10303000EFD02FE20247FD576310F70297D7010048
:103040009387473A9C439107BE8517D50100130526
:103050006555EFD06FD519A897D70100938707560C
:103060009C430247BA973ECC6245893AEFD00FBAEB
:10307000FD3BF933924789CB97D701009387873679
:103080009C43B84F924798C397D7010093878735E1
:103090009C43F84F85476314F70002CE31A897D7B9
:1030A0000100938727349C43B44F22471347F7FF0F
:1030B000758FB8CF85473ECE97D70100938787326B
:1030C0009C4323AE07046533F2473E85B250456109
:1030D0008280797106D62AC62EC432C236C0854790
:1030E0003ECEB24781E77370043001A0B2473ECCB8
:1030F000813B824789C7E247B84F824798C3E2477E
:10310000FC4F3ECAE2470947F8CF1247914763EEAA
:10311000E70492471397270097D70100938707EF9B
:10312000BA97984397D70100938747EEBA9782875B
:10313000E247B84FA2475D8FE247B8CF3DA0E247D4
:10314000BC4F13871700E247B8CF05A0E2472247DC
:10315000B8CF21A8524789476306F700E2472247C4
:10316000B8CF21A002CE11A0010052478547631AB3
:10317000F706E24791073E85EFD0AFCDE247D8573B
:1031800097D701009387C7439C4363F9E700E24761
:10319000D85797D701009387A74298C3E247D857DB
:1031A000BA878A07BA978A0717D701001307472DEE
:1031B0003E97E2479107BE853A85EFD0EFBEE247E2
:1031C0009C5781C77370043001A0E247D85797D746
:1031D0000100938727219C43DC5763F4E700EFD07D
:1031E000EFA27131F2473E85B2504561828039715C
:1031F00006DE2ACE2ECC32CA36C83AC685473ED61F
:10320000F24781E77370043001A0F2473ED4EFD05B
:10321000CFADAA873ED2C24789C7A257B84FC2478F
:1032200098C3A257FC4F3ED0A2570947F8CF524748
:10323000914763EEE704D2471397270097D7010021
:10324000938707DEBA97984397D70100938747DDA6
:10325000BA978287A257B84FE2475D8FA257B8CF7F
:103260003DA0A257BC4F13871700A257B8CF05A0A7
:10327000A2576247B8CF21A8025789476306F700D3
:10328000A2576247B8CF21A002D611A00100025771
:103290008547631DF708A2579C5781C77370043098
:1032A00001A097D70100938767339C43A1EBA257F6
:1032B00091073E85EFD0EFB9A257D85797D70100B5
:1032C000938707309C4363F9E700A257D85797D7F5
:1032D00001009387E72E98C3A257D857BA878A0769
:1032E000BA978A0717D70100130787193E97A25785
:1032F0009107BE853A85EFD02FAB11A8A257E10701
:10330000BE8517D5010013052527EFD0EFA9A257D9
:10331000D85797D701009387E70C9C43DC5763F796
:10332000E700B24781C7B247054798C392573E8529
:10333000EFD0AF9AB2573E85F25021618280797109
:1033400006D62AC62EC4B24781E77370043001A0A6
:10335000B2473ECEEFD06F99AA873ECCF247FC4FE2
:103360003ECAF2470947F8CFF247BC4F1387170010
:10337000F247B8CF52478547631DF708F2479C577D
:1033800081C77370043001A097D701009387072588
:103390009C43A1EBF24791073E85EFD08FABF247FC
:1033A000D85797D701009387A7219C4363F9E7007B
:1033B000F247D85797D701009387872098C3F247E1
:1033C000D857BA878A07BA978A0717D70100130711
:1033D000270B3E97F2479107BE853A85EFD0CF9CE9
:1033E00011A8F247E107BE8517D501001305C518DE
:1033F000EFD08F9BF247D85797D70100938787FE6E
:103400009C43DC5763F7E700A24781C7A247054703
:1034100098C3E2473E85EFD04F8C0100B250456122
:103420008280797106D62AC6B2473ECCE24799E738
:1034300097D70100938707FB9C4311A0E2473ECC3E
:103440000134E247F84F89476318F700E24723AE9B
:10345000070485473ECE11A002CE113CF2473E85BF
:10346000B25045618280011106CE02C61D2B97D74E
:1034700001009387E7199C439DC381480148814718
:10348000094781461306004097D50100938585BA08
:10349000170500001305051BEFE0AF852AC6B247EC
:1034A00081E77370043001A0B2473E85F2400561A8
:1034B0008280397106DE2ACE2ECC32CA36C83AC690
:1034C000E24799E302D62DA81305C002EF00302A87
:1034D0002AD6B25795C7F121B257724798C3B2574F
:1034E000624798CFB2575247D8CFB257424798D386
:1034F000B2573247D8D3B25791073E85EFD0CF8924
:10350000E24781E77370043001A0B2573E85F25064
:1035100021618280397106DE2ACE2ECC32CA36C8AD
:103520003AC602D6F24781E77370043001A097D7FC
:1035300001009387E70D9C43B5CBE2473ED0D247CD
:103540003ED2F2473ED46247954763C4E704EFF0AA
:10355000AFF22A8789476310F70297D70100938754
:10356000270B9C43181081463246BA853E85EFD022
:103570002FBF2AD625A897D70100938767099C43B8
:10358000181081460146BA853E85EFD06FBD2AD618
:1035900031A897D701009387A7079C43181081464D
:1035A0004246BA853E85EFD08FF22AD6B2573E8585
:1035B000F2502161828001112AC6B2473ECEB24745
:1035C00081E77370043001A0F2479C433E8505619A
:1035D0008280797106D62AC62EC497D701009387B8
:1035E000A7029C43DC47DC473ECEF24791073E856D
:1035F000EFD02F86F247D84F8547631BF702F2477B
:10360000984FB247BA97B2462246BE857245B92254
:103610002A878547631EF700014781463246814568
:103620007245CD3D2ACCE24781E77370043001A09A
:10363000F247DC53724582970100B25045618280A7
:10364000797106D62AC63C083E8541282ACEE24733
:10365000BE85724519206922FDB7797106D62AC642
:103660002EC4EFE06FF93C083E8545282ACEE2479C
:10367000B9EFA24799EB3247F24763E8E700EFE082
:103680006FF9F2453245B137A9A0A24781CF97D74C
:1036900001009387A7F79C439C4393B7170093F7C8
:1036A000F70F3EC497D70100938787F694433247BC
:1036B000F247B307F7402246BE853685EFD0FFDDDF
:1036C000EFE04FF5AA8791E7EFC05FD419A0EFE0D4
:1036D0006FF40100B2504561828001112AC697D76C
:1036E0000100938767F29C439C4393B7170093F7BD
:1036F000F70F3E87B24798C3B2479C4391EB97D7E9
:103700000100938767F09C43DC479C433ECE11A0A9
:1037100002CEF2473E8505618280797106D62AC6BF
:10372000EFE01F842ACE97D701009387A7EE9C4332
:1037300072476377F700692AB247054798C321A00B
:10374000B24723A0070097D701009387A7EC7247E1
:1037500098C3F2473E85B25045618280797106D6A2
:103760002AC62EC432C236C002CEB2472247D8C3C0
:10377000B247324798CB2247924763E8E7021247A5
:1037800082471D8FB2479C4F6365F70085473ECE49
:1037900099A097D70100938767E79843B2479107AD
:1037A000BE853A85EFC05FE43DA01247824763794A
:1037B000F700224782476365F70085473ECE21A880
:1037C00097D70100938747E49843B2479107BE8596
:1037D0003A85EFC07FE1F2473E85B2504561828075
:1037E000797106D6D9A0A24763C0070CC2473ECE66
:1037F000F247DC4B91C7F24791073E85EFC07FE56A
:103800005C003E85193F2ACCA2472547636FF70825
:103810001397270097D7010093874782BA97984359
:1038200097D7010093878781BA9782873247F247FB
:103830009C4FBA973247BA866246BE857245393F79
:103840002A8785476313F706F247DC537245829750
:10385000F247D84F8547631AF7043247F2479C4F27
:10386000BA97014781463E868145724565312ACA2D
:10387000D24785EF7370043001A03247F24798CFEA
:10388000F2479C4F81E77370043001A0F247984FD4
:10389000E247BA97E2466246BE857245C13531A01D
:1038A0007245EF00C07F11A0010097D701009387F8
:1038B00027D69C43380081460146BA853E85EFD025
:1038C0006FD8AA87E39107F20100B2504561828068
:1038D000797106D671A097D701009387E7D29C43F0
:1038E000DC479C433ECC97D701009387E7D19C43AC
:1038F000DC47DC473ECAD24791073E85EFC07FD503
:10390000D247DC5352458297D247D84F8547631937
:10391000F704D2479C4F6247BA973EC84247E247F6
:1039200063F4E702D2474247D8C3D247524798CB05
:1039300097D70100938747CD9843D2479107BE851B
:103940003A85EFC07FCA29A8014781466246814572
:103950005245C9362AC6B24781E77370043001A0C8
:1039600097D70100938747CA9C439C43ADF797D7ED
:103970000100938767C99C433ECE97D70100938788
:10398000E7C8984397D70100938707C898C397D78C
:1039900001009387A7C7724798C30100B2504561E1
:1039A0008280411106C6EFF0AFC997D70100938717
:1039B00027C69C43C9E717D50100130565C2EFC0B0
:1039C0007FBA17D501001305E5C2EFC0BFB997D77D
:1039D0000100938767C317D70100130767C098C317
:1039E00097D70100938787C217D70100130787C0B5
:1039F00098C30146B1451145EFC0FFD52A8797D737
:103A000001009387E7C098C397D70100938747C009
:103A10009C4381E77370043001A097D7010093871E
:103A200027BF9C4389CF97D70100938767BE9C43EC
:103A300097C50100938505633E85EFD05F9CEFF04D
:103A40000FC30100B24041018280797106D62AC6B7
:103A5000B2473ECEB24781E77370043001A0EFF069
:103A60002FBEF247DC4BB337F00093F7F70F3ECC95
:103A7000EFF0EFBFE2473E85B25045618280797139
:103A800006D62AC6B2473ECEB24781E773700430ED
:103A900001A0EFF0EFBAF2479C533ECCEFF02FBD00
:103AA000E2473E85B25045618280797106D62AC6CA
:103AB0002EC4B2473ECEB24781E77370043001A0F6
:103AC000EFF00FB8F247224798D3EFF04FBA01005A
:103AD000B25045618280011106CE714549292AC63E
:103AE000B24789CBB24723A00700B24791073E8572
:103AF000EFC05FA7B2473E85F24005618280397111
:103B000006DE2AC62EC432C236C0B2473ED402D226
:103B10001247B70700FFF98F81C77370043001A007
:103B2000924781E77370043001A0EFF0EF94AA8709
:103B300099E3824799E3854711A0814781E7737034
:103B4000043001A0EFE04FABA2579C433ED0A2450A
:103B5000324585240257A2475D8F9247F98F12475D
:103B60006310F7020257A247D98F3ED6A257984357
:103B7000924793C7F7FF7D8FA25798C302C025A035
:103B8000824799CFA257938647001247B70700058F
:103B9000D98F0246BE853685EFE03F8902D621A047
:103BA000A2579C433ED6EFE0EFA62ACE8247B1CB88
:103BB000F24799E3EFC09F85EFF06FAF2AD63257F7
:103BC000B7070002F98F85EBEFF08FA7A2579C4350
:103BD0003ED632579247F98F1247631AF700A25721
:103BE0009843924793C7F7FF7D8FA25798C3EFF092
:103BF0000FA885473ED23257B7070001FD17F98F4E
:103C00003ED6B2573E85F250216182805D7186C6F4
:103C10002ACE2ECC32CA36C83AC6F2473EDA02DC89
:103C200002D8F24781E77370043001A06247B707FA
:103C300000FFF98F81C77370043001A0E24781E76C
:103C40007370043001A0EFF02F83AA8799E3B24785
:103C500099E3854711A0814781E77370043001A083
:103C6000EFE08F99D2579C433ED64246E24532550B
:103C700075242AD4A25799CFB2573EDE02C6D24746
:103C8000A9CBD2579843E24793C7F7FF7D8FD2570E
:103C900098C381A0B24781E7B2573EDE1DA8D24744
:103CA00091C76257B7070001D98F3EDCC24791C761
:103CB0006257B7070004D98F3EDCD257938647007E
:103CC0006247E257D98F3246BE853685EFE0EFF581
:103CD00002DEEFE02F942AD2B247B9CB925799E394
:103CE000EFC0CFF2EFF0AF9C2ADE7257B7070002A9
:103CF000F98F8DEBEFF0CF94D2579C433EDE4246D6
:103D0000E2457255212CAA8799CBD24789CBD2574D
:103D10009843E24793C7F7FF7D8FD25798C3EFF0E0
:103D20000F9502D87257B7070001FD17F98F3EDED5
:103D3000F2573E85B64061618280797106D62AC607
:103D40002EC4B2473ECEB24781E77370043001A063
:103D50002247B70700FFF98F81C77370043001A0B5
:103D6000EFF00F8EF2479C433ECCF2479843A247B8
:103D700093C7F7FF7D8FF24798C3EFF04F8FE2476D
:103D80003E85B25045618280797106D62AC6B24717
:103D90003ECEEFC08FF5AA873ECCF2479C433ECA89
:103DA000E2473E85EFC06FF3D2473E85B250456192
:103DB00082805D7186C62AC62EC402DCB2473ED818
:103DC00002DAB24781E77370043001A02247B707D7
:103DD00000FFF98F81C77370043001A0C2579107AB
:103DE0003ED6B257A1073ED4EFE00F81B257DC4771
:103DF0003EDEC2579843A2475D8FC25798C3BDA805
:103E0000F257DC433ED2F2579C433ED002DA0257CF
:103E1000B70700FFF98F3ECE0257B7070001FD1725
:103E2000F98F3ED07247B7070004F98F89EBC2576C
:103E300098438257F98F89CF85473EDA11A8C25738
:103E400098438257F98F02576314F70085473EDA8B
:103E5000D2579DC37247B7070001F98F89C76257D0
:103E60008257D98F3EDCC2579843B7070002D98FDB
:103E7000BE857255EFE00FF992573EDE7257A2579A
:103E8000E310F7F8C2579843E25793C7F7FF7D8FC7
:103E9000C25798C3EFD01FF8C2579C433E85B64027
:103EA00061618280797106D62AC6B2473ECEF2475A
:103EB00091073ECCEFD05FF40DA0E247D847E24730
:103EC000A1076315F7007370043001A0E247DC47D7
:103ED000B70500023E85EFE0EFF2E2479C43F1FFB9
:103EE0007245752AEFD01FF30100B2504561828000
:103EF000011106CE2AC62EC4A24532455D3D010001
:103F0000F24005618280011106CE2AC62EC4A24568
:103F1000324525350100F2400561828001112AC633
:103F20002EC432C202CE924781EB3247A247F98FAC
:103F300081CF85473ECE09A83247A247F98F224755
:103F40006314F70085473ECEF2473E8505618280C7
:103F500001112AC6B2473ECCB24799E302CE21A056
:103F6000E2479C4F3ECEF2473E8505618280397123
:103F700006DE2AC602D2EFD03FE8975703009387A8
:103F8000A76A9C4381EB5522975703009387C76923
:103F9000054798C3B24789CFA1473E87B247BA9732
:103FA0003EC6B2478D8B89C7B247F19B91073EC68B
:103FB000B247F9CB3247E567ED1763E7E70C975750
:103FC0000300938767653ED4975703009387C764C0
:103FD0009C433ED631A0B2573ED4B2579C433ED606
:103FE000B257DC43324763F5E700B2579C43E5F72D
:103FF0003257975703009387A7626307F708A257C2
:104000009C432147BA973ED2B2579843A25798C3D0
:10401000B257D843B247B307F74021470607637842
:10402000F7043257B247BA973ECEB257D843B24799
:104030001D8FF247D8C3B2573247D8C3F247DC438B
:104040003ECC975703009387275D3ED021A082572F
:104050009C433ED082579C43DC436247E3E9E7FE42
:1040600082579843F24798C38257724798C397C7BD
:104070000100938767389843B257DC431D8F97C779
:1040800001009387673798C3EFD0DFD8925799E341
:10409000EF00303292573E85F25021618280797173
:1040A00006D62AC6B2473ECCB247BDC3A147B30726
:1040B000F0406247BA973ECCE2473ECAEFD0DFD32A
:1040C000D247DC433EC8975703009387E7543ECE60
:1040D00021A0F2479C433ECEF2479C43DC4342473B
:1040E000E3E9E7FEF2479843D24798C3F2475247C5
:1040F00098C3D247D84397C701009387E72F9C43C3
:104100003E9797C701009387272F98C3EFD09FD082
:104110000100B2504561828097C701009387C72D87
:104120009C433E85828001008280411197C7010037
:104130009387C74EF19B3EC6975703009387C74DA1
:10414000324798C3975703009387074D23A2070070
:10415000975703009387C74C65677117D8C3975764
:1041600003009387E74B23A00700B2473EC4A24752
:1041700065677117D8C3A247175703001307474A4B
:1041800098C301004101828001112AC62EC432C2A7
:10419000A2473ECEB2473ECC3247A247D98F8D8B45
:1041A000A1E319A8F2479843E24798C3E247910771
:1041B0003ECCF24791073ECE9247F5173247BA9769
:1041C0006247E361F7FE29A87247930717003ECEC6
:1041D000E2479386170036CC034707002380E700A9
:1041E00032479247BA976247E360F7FEB2473E858F
:1041F0000561828001112AC62EC432C2324792471D
:10420000D98F8D8B9DEFA24793F7F70F3ECAD24708
:10421000A2075247D98F3ECAD247C2075247D98F09
:104220003ECAB2473ECE39A0F247138747003ACE86
:10423000524798C332479247BA977247E366F7FEF0
:104240001DA0B2473ECC11A8E247138717003ACC15
:1042500022471377F70F2380E70032479247BA9738
:104260006247E363F7FEB2473E8505618280011134
:104270002AC6B2473ECE21A0F24785073ECEF2477E
:1042800083C70700F5FB7247B247B307F7403E8587
:104290000561828001112AC62EC4B2471387170018
:1042A0003AC683C70700A30FF100A2471387170080
:1042B0003AC483C70700230FF1008347F10199C770
:1042C0000347F1018347E101E309F7FC0347F101EB
:1042D0008347E101B307F7403E8505618280011104
:1042E0002AC62EC4B2473ECE0100224793071700CC
:1042F0003EC4F2479386170036CE0347070023805B
:10430000E70083C70700F5F3B2473E850561828069
:1043100001112AC602CE02CC21A0B24785073EC6B3
:10432000B24703C7070093070002E308F7FEB2474E
:1043300003C707009307D0026309F700B24703C71A
:1043400007009307B0026311F704B24783C7070061
:10435000938737FD93B7170093F7F70F3ECCB2471B
:1043600085073EC615A07247BA878A07BA9786079F
:104370003ECEB247138717003AC683C7070093871C
:1043800007FD7247BA973ECEB24783C70700E1FFE9
:10439000E24789C7F247B307F04011A0F2473E85D4
:1043A0000561828001112AC69757030093878729E8
:1043B0009C4393861700175703001307A72814C3BD
:1043C00032471377F70F975603009386A62BB697BD
:1043D0002380E7003247A947630BF7009757030094
:1043E000938747269843930700046315F70497576C
:1043F0000300938727293ECE05A8F24713871700AD
:104400003ACE03C70700B70710F0938707F098C3A9
:1044100097570300938707239C431387F7FF97570A
:1044200003009387272298C3975703009387872118
:104430009C43E1F781473E85056182804D712326CB
:104440001114232481142322911423202115232EB7
:104450003113232C4113232A51132ACE2ECC32C8D8
:1044600036CA3AC63EC442C223260112B2473E8A29
:10447000814AC24752485286D6863E85C285EF1091
:10448000A03AAA872E883E86C2868327C112138748
:1044900017002326E11232878A07141AB69723AE33
:1044A000E7EEB2473E848144D247268763E8E702BD
:1044B000D24726876396E700C247228763E0E70278
:1044C000B2473E8981494A86CE864245D245EF00B1
:1044D000F057AA872E883EC842CA49BF010029A0CA
:1044E000F247E24512458297A2471387F7FF3AC485
:1044F0000327C112E346F7FE25A88327C1128A07C6
:10450000181ABA9703A7C7EF8327C1128A07141A8C
:10451000B69783A6C7EFA54763F5D7009307700545
:1045200019A093070003BA977247E2453E850297A8
:104530008327C1121387F7FF2326E112E34FF0FA16
:1045400001008320C114032481148324411403290E
:1045500001148329C113032A8113832A4113716132
:10456000828041112AC62EC4A2460547635ED70049
:10457000B2479C439D07E19B93868700324714C353
:1045800003A847009C4335A0224719CB3247184364
:1045900013064700B24690C21843BA87014811A8D3
:1045A0003247184313064700B24690C21843BA87F1
:1045B00001483E85C2854101828041112AC62EC430
:1045C000A2460547635ED700B2479C439D07E19B27
:1045D00093868700324714C303A847009C4305A86D
:1045E000224701CF3247184313064700B24690C214
:1045F0001843BA877D873A8819A8324718431306AB
:104600004700B24690C21843BA877D873A883E85F4
:10461000C28541018280397106DE22DC26DA2AC693
:104620002EC432C236C011A86307042492478507FE
:104630003EC2B247A24522858297924783C70700B0
:104640003E8493075002E311F4FE924785073EC271
:1046500092473EC893070002A30BF100FD573ECEE0
:10466000FD573ECC02D09247138717003AC283C74A
:1046700007003E849307D4FD130750056364F71EBB
:104680001397270097C701009387C79EBA9798434F
:1046900097C701009387079EBA9782879307D00236
:1046A000A30BF100C9B793070003A30BF10065BF8B
:1046B00002CC6247BA878A07BA978607A297938780
:1046C00007FD3ECC924783C707003E849307F00264
:1046D00063D687029307900363C2870292478507D8
:1046E0003EC2C1BF8247138747003AC09C433ECCBD
:1046F00039A0F247E3D907F602CEB5B70100F24779
:10470000E3D307F6E2473ECEFD573ECCA9BF825722
:1047100085073ED089BF8247138747003AC09C4334
:104720003247A2453E850297B1A2824713874700D0
:104730003AC0844389E497C4010093842493F247E8
:104740006357F004034771019307D0026301F70434
:10475000E247BE852685EF00302D2A87F247998FE4
:104760003ECE11A8834771013247A2453E8502978C
:10477000F247FD173ECEF247E346F0FE09A8B247E6
:10478000A245228582978504F247FD173ECE83C756
:1047900004003E841DC0E247E3C307FEE247FD1765
:1047A0003ECCE247E3DD07FC09A8B247A24513056A
:1047B00000028297F247FD173ECEF247E347F0FE34
:1047C00055A88A8782553E85CD3BAA872E883ED440
:1047D00042D6A2573258C28763D90702B247A245D0
:1047E0001305D0028297A255325681470148B386FD
:1047F000B740368533B5A7003307C840B307A74095
:104800003E87B6873A883ED442D6A9473ED21DA8F5
:10481000A9473ED215A0A1473ED239A885473ED030
:10482000B247A245130500038297B247A24513057C
:1048300080078297C1473ED28A8782553E851533CD
:104840002AD42ED61257834771013E88F24722564A
:10485000B256A2453245DD3631A8B247A24522857F
:10486000829709A8B247A245130550028297C24712
:104870003EC20100D9B30100F2506254D25421610A
:10488000828041112AC6B70710F0938707F232479A
:1048900098C301A05D7106D62AC62EDA32DC36DE58
:1048A000BAC0BEC2C2C4C6C69C0891173ECEF2476B
:1048B000BE8632468145170500001305E5AEA13BD3
:1048C00081473E85B2506161828001112AC62EC4A3
:1048D0001EC2A2473ECEF2479C4332471377F70FE2
:1048E0002380E700F2479C4313871700F24798C3E1
:1048F0000100056182801D7106DE2AC62EC4B2C485
:10490000B6C6BAC8BECAC2CCC6CE9C103ED25C08DF
:104910004C0817060000130686FB7D779346F7FFC9
:104920000565130505803388A5003378E800136812
:10493000783B23A007013295698F13677733D8C37B
:1049400033F7D5009315470137870300130737392D
:104950004D8F98C73377D60093164701370703006A
:1049600013077706558FD8C70F100000B2473ED601
:104970009C10A1173ED422575C083E857C00BA8665
:104980002246BE854939B24723800700B2473E8799
:10499000B257B307F7403E85F2502561828041113E
:1049A000370510F0130545F408412AC6370510F005
:1049B000130505F408412AC4370510F0130545F422
:1049C0000841B248E39EA8FC32452A83814313176D
:1049D000030081462245AA850146B3E7B600336845
:1049E000C700370710F0130587F49305007D0146D3
:1049F000B386B700B688B3B8F8003307C800B387EA
:104A0000E8003E87B6873A881CC1232205010100D1
:104A100041018280411106C659379307000873A0EF
:104A200047300100B24041018280011106CE2AC602
:104A300017B5010013058579EFF0DFE50100F240BD
:104A400005618280011106CE2AC617B50100130543
:104A50006578EFF03FE40100F240056182807971F2
:104A600006D62AC602CE29A00100F24785073ECE0F
:104A70007247856793877738E3D8E7FE17B501005B
:104A80001305C575EFF01FE1F1BF411106C62D2AD0
:104A90000100B24041018280011106CE02C6EF0042
:104AA000C0702A878547630CF70017B5010013050E
:104AB0006573EFF03FDEB24793E727003EC6B2478B
:104AC0003E85F24005618280011106CE02C6753F27
:104AD0001707000013076704814605469305400643
:104AE00017B501001305C571EFE0BF9C2AC6B24798
:104AF00099CBEFD0EFC6AA87014781463E86854510
:104B00003245EFE03FA102C4EFD02FA581473E859B
:104B1000F24005618280797106D62AC697C70100E6
:104B20009387878C9C431387470697C70100938719
:104B3000A78B98C397C701009387478B9C43138724
:104B4000470697C701009387678A98C397C70100F4
:104B50009387878998438567938777BB63D5E704F5
:104B600097C70100938747889843FD7793878744C9
:104B70003E9797C701009387278798C3313F2ACE76
:104B8000F24799EB97C70100938747869843896757
:104B90009387773263DBE700F2473E85EFF07FCE05
:104BA000EFD08FA321A0010011A00100B2504561F8
:104BB00082807370043001A00100828041112AC6F6
:104BC0002EC47370043001A0411106C60146914500
:104BD0001545EFB05FB82A8797570300938787AED4
:104BE00098C3975703009387E7AD9C4397B501009F
:104BF0009385C5613E85EFC09F808148014881470C
:104C00000D4781461306004097B501009385056165
:104C1000170500001305C503EFC0BF8D814801488B
:104C200097570300938747AA094781461306004018
:104C300097B501009385055F1705000013058542B0
:104C4000EFC03F8B0100B24041018280397106DE26
:104C50002AC602D041A082572947B317F7003ED693
:104C6000EFE00F9EEFD0CFAF2AD497570300938782
:104C700067A59C43780881463256BA853E85EFB0D9
:104C80001FF2AA8799C7975703009387A7A40547E0
:104C900098C3EFD0EFAC2A87A257B307F7403ED2B4
:104CA000EFE0EF9C1257B2576378F7009757030075
:104CB000938747A2054798C3B257B107125763F8C5
:104CC000E700975703009387E7A0054798C38257EB
:104CD00085073ED002579147E3DFE7F602D015A8DB
:104CE000975703009387079E9C43181081460146FF
:104CF000BA853E85EFB03FDD2A8785476308F70018
:104D0000975703009387079D054798C382578507E8
:104D10003ED002579147E3D5E7FC02D041A082572D
:104D20002947B317F7003ED6EFE08F91EFD04FA39E
:104D30002AD4975703009387E7989C43181081461D
:104D40003256BA853E85EFB01FD8AA8799C79757C4
:104D5000030093872798054798C3EFD06FA02A8751
:104D6000A257B307F7403ED2EFE06F901257B25709
:104D70006378F700975703009387C795054798C353
:104D8000B257B107125763F8E700975703009387AC
:104D90006794054798C3825785073ED002579147CD
:104DA000E3DFE7F6975703009387079323A00700F5
:104DB00097570300938747919C433E85EFC07FE35D
:104DC00021A05145EFC01FA6975703009387C790B6
:104DD000984393075005E316F7FE5145EFC09FA493
:104DE000975703009387478F23A0070002D0C1A0E5
:104DF000975703009387078D9C43780881460146A7
:104E0000BA853E85EFB0BFD92A8785476308F7008A
:104E1000975703009387078C054798C3975703005C
:104E20009387478A9C43181081460146BA853E8580
:104E3000EFB07FC92A8785476308F70097570300BB
:104E400093874789054798C3975703009387C78877
:104E50009843930750056318F7009757030093870B
:104E60006787054798C3975703009387E7859C4357
:104E700095453E85EFC07FB1975703009387C7855F
:104E80009843930750056318F700975703009387DB
:104E90006784054798C3975703009387E7829C432D
:104EA00089453E85EFC07FAE825785073ED00257C9
:104EB0009147E3DFE7F221A05145EFC0BF96975736
:104EC000030093876781984393075005E316F7FE25
:104ED0005145EFC03F95974703009387E77F23A095
:104EE000070002D015A8974703009387A77D9C432E
:104EF000780881460146BA853E85EFB05FCA2A87A9
:104F000085476308F700974703009387A77C054709
:104F100098C3825785073ED002579147E3D5E7FCF7
:104F2000974703009387477A9C433E85EFC07FCC29
:104F300021A05145EFC01F8F974703009387C77982
:104F4000984393075005E316F7FE5145EFC09F8D38
:104F5000974703009387477823A0070002D0C1A09A
:104F600097470300938707769C43181081460146B4
:104F7000BA853E85EFB03FB52A8785476308F700BD
:104F80009747030093870775054798C39747030022
:104F9000938747739C43780881460146BA853E85CE
:104FA000EFB0FFBF2A8785476308F70097470300E4
:104FB00093874772054798C3974703009387C77144
:104FC0009843930750056318F700974703009387AA
:104FD0006770054798C3974703009387E76E9C4324
:104FE00095453E85EFC07F9A974703009387C76E2C
:104FF0009843930750056318F7009747030093877A
:10500000676D054798C3974703009387E76B9C43F9
:1050100089453E85EFC07F97825785073ED002576E
:105020009147E3DFE7F221A05145EFC0AFFF97477B
:1050300003009387676A984393075005E316F7FECA
:105040005145EFC02FFE97470300938727689C4385
:1050500013871700974703009387476798C3D5BE08
:10506000797106D62AC60145EFC09FA6EFD05FDD55
:10507000EFC01FEF2ACE02CA974703009387C76588
:105080001307500598C3974703009387A7639C4372
:10509000580881461306F00ABA853E85EFB0BFA2D4
:1050A000AA8799C7974703009387C762054798C3A4
:1050B000EFC01FEB2A87F247B307F7403ECCEFD093
:1050C0001FDB62479307E00A63E8E70097470300A6
:1050D00093874760054798C362479307B00B63F80F
:1050E000E700974703009387E75E054798C3974714
:1050F00003009387675E1307500598C30145EFC00F
:105100003F9DEFD0FFD3EFC0BFE52ACE9747030006
:105110009387875C1307500598C3974703009387CD
:10512000675A9C43580881461306F00ABA853E85A3
:10513000EFB0FFA6AA8799C79747030093878759BF
:10514000054798C3EFC0DFE12A87F247B307F7406E
:105150003ECCEFD0DFD162479307E00A63E8E70077
:105160009747030093870757054798C362479307FC
:10517000B00B63F8E700974703009387A7550547EF
:1051800098C397470300938727551307500598C383
:10519000974703009387C7539C431387170097478C
:1051A00003009387E75298C37DBD411185473EC6F2
:1051B0009747030093878751984397470300938746
:1051C000E7519C436313F70002C697470300938798
:1051D0002750984397470300938787509C43631356
:1051E000F70002C6974703009387C74E9843854749
:1051F0006313F70002C6974703009387674D9843F0
:10520000974703009387C74D98C397470300938739
:10521000E74B9843974703009387474C98C3B2479F
:105220003E85410182800000B305B500930705006B
:105230006386B70003C70700631607003385A740DE
:1052400067800000938717006FF09FFE130101FD38
:1052500023229102232A51012326110223248102B1
:1052600023202103232E3101232C41012328610116
:105270002326710123248101232291012320A101EE
:10528000930A050093840500639E06381304060004
:105290009309050017B90100130949F963F8C5120C
:1052A000B7070100138B05006378F6101307F00FA2
:1052B0003337C70013173700B357E6003309F90037
:1052C000834609003387E60093060002B386E64072
:1052D000638C0600B394D40033D7EA003314D600AD
:1052E000336B9700B399DA00935A040193850A004F
:1052F00013050B00EF00902A1309050093850A009F
:10530000931B040113050B00EF00D02493DB0B016A
:10531000930405009305050013850B00EF00D020D2
:105320001319090193D70901B367F900138A04001F
:1053300063FEA700B3878700138AF4FF63E8870042
:1053400063F6A700138AE4FFB3878700B384A740FE
:1053500093850A0013850400EF005024130905000B
:1053600093850A0013850400EF00D01E939909016C
:1053700093040500930505001319090113850B001B
:1053800093D90901EF00501AB3693901138604005B
:1053900063FCA900B30934011386F4FF63E68900B6
:1053A00063F4A9001386E4FF13140A013364C400F4
:1053B000130A00006F000013B70700011307000174
:1053C000E36CF6EE130780016FF01FEF138A0600FF
:1053D000631A06009305000013051000EF009017F4
:1053E00013040500B7070100637EF4129307F00F62
:1053F00063F48700130A8000B35744013309F900AE
:10540000034709009306000233074701B386E640CD
:1054100063940612B3848440130A1000135B0401E2
:1054200093050B0013850400EF00501713090500C6
:1054300093050B0013850400931B0401EF009011EA
:1054400093DB0B01930405009305050013850B0006
:10545000EF00900D1319090193D70901B367F90003
:10546000938A040063FEA700B3878700938AF4FF42
:1054700063E8870063F6A700938AE4FFB387870099
:10548000B384A74093050B0013850400EF001011AF
:105490001309050093050B0013850400EF00900B22
:1054A0009399090193040500930505001319090157
:1054B00013850B0093D90901EF001007B369390177
:1054C0001386040063FCA900B30934011386F4FFBA
:1054D00063E6890063F4A9001386E4FF13940A01CC
:1054E0003364C4001305040093050A008320C1023D
:1054F0000324810283244102032901028329C1017B
:10550000032A8101832A4101032B0101832BC1005E
:10551000032C8100832C4100032D010013010103A2
:1055200067800000B7070001130A0001E366F4EC8E
:10553000130A80016FF05FEC3314D40033DAE40017
:10554000B399DA0033D7EA00935A0401B394D40034
:1055500093850A0013050A00336B9700EF001004CF
:105560001309050093850A0013050A00931B040123
:10557000EF00407E93DB0B019304050093050500CB
:1055800013850B00EF00407A1319090113570B0123
:105590003367E900138A0400637EA700330787009E
:1055A000138AF4FF636887006376A700138AE4FF19
:1055B00033078700B304A74093850A0013850400CE
:1055C000EF00C07D1309050093850A0013850400D0
:1055D000EF004078930405009305050013850B0048
:1055E000EF00807413170B011357070113190901FA
:1055F000B367E9001387040063FEA700B387870041
:105600001387F4FF63E8870063F6A7001387E4FFBE
:10561000B3878700131A0A01B384A740336AEA00EC
:105620006FF0DFDF63ECD51EB707010063F4F6040B
:105630001307F00FB335D7009395350033D7B60075
:1056400097B70100938787BEB387E70003C70700BA
:10565000130A00023307B700330AEA4063160A024E
:1056600013041000E3E096E833B6CA0013441600B2
:105670006FF05FE7B707000193050001E3E0F6FC78
:10568000930580016FF09FFBB35CE600B396460183
:10569000B3ECDC0033D4E40093DB0C01B39744019A
:1056A00033D7EA0093850B0013050400336BF70032
:1056B000B3194601EF00806E1309050093850B00B6
:1056C00013050400139C0C01EF00C068135C0C016F
:1056D000930405009305050013050C00EF00C0645A
:1056E0001319090113570B013367E90013840400F0
:1056F000637EA700330797011384F4FF6368970163
:105700006376A7001384E4FF33079701B304A7402F
:1057100093850B0013850400EF0040681309050012
:1057200093850B0013850400EF00C062930405000D
:105730009305050013050C00EF00005F93170B01A4
:105740001319090193D70701B367F9001386040001
:1057500063FEA700B38797011386F4FF63E8970100
:1057600063F6A7001386E4FFB387970113140401BF
:10577000B70B01003364C4001389FBFF337D2401A0
:1057800033F92901B384A7409305090013050D00DF
:10579000EF008059935C040193050900130B050089
:1057A00013850C00EF00405893D90901130C050034
:1057B0009385090013850C00EF00005713090500BD
:1057C0009385090013050D00EF0000563305850190
:1057D00093570B013385A700637485013309790161
:1057E00093570501B387270163E6F402E392F4BC03
:1057F000B70701009387F7FF3375F500131505010F
:10580000337BFB0033964A0133056501130A000020
:10581000E37AA6CC1304F4FF6FF09FB9130A0000DB
:10582000130400006FF01FCC130101FB232481043B
:1058300023229104232E31032322910323261104D2
:1058400023202105232C4103232A5103232861030C
:1058500023267103232481032320A103232EB101D6
:10586000930C05009389050013040500938405003B
:10587000639E062613090600138A060097BA0100E4
:10588000938ACA9A63F4C514B70701006376F612C7
:105890009307F00F63F4C700130A8000B357460163
:1058A000B38AFA0003C70A00130500023307470151
:1058B000330AE540630C0A00B395490133D7EC0085
:1058C00033194601B364B70033944C01935A09016C
:1058D00093850A0013850400EF00404C93090500EE
:1058E00093850A00131B090113850400EF0080460D
:1058F000135B0B019305050013050B00EF00C0427D
:105900009399090193570401B3E7F90063FAA700DB
:10591000B387270163E6270163F4A700B387270154
:10592000B384A74093850A0013850400EF00004765
:105930009309050093850A0013850400EF00804158
:1059400013140401930505009399090113050B0035
:1059500013540401EF00403D33E48900637AA4004E
:1059600033042401636624016374A4003304240116
:105970003304A44033554401930500008320C1043F
:105980000324810483244104032901048329C103DE
:10599000032A8103832A4103032B0103832BC102C2
:1059A000032C8102832C4102032D0102832DC101AE
:1059B0001301010567800000B7070001130A000109
:1059C000E36EF6EC130A80016FF05FED631A0600D8
:1059D0009305000013051000EF00C0371309050000
:1059E000B7070100637AF90E9307F00F63F42701FC
:1059F000130A8000B3574901B38AFA0003C70A00AB
:105A000013050002B384294133074701330AE540F7
:105A1000E30E0AEA33194901B3DAE900B395490103
:105A200033D7EC0093540901336BB70013850A0098
:105A300093850400EF0080369309050093850400E8
:105A4000931B090113850A00EF00C03093DB0B01A3
:105A50009305050013850B00EF00002D93990901B4
:105A600093570B01B3E7F90033944C0163FAA70095
:105A7000B387270163E6270163F4A700B3872701F3
:105A8000B38AA7409385040013850A00EF00003114
:105A9000930905009385040013850A00EF00802B0D
:105AA0009305050013850B00EF00002893150B01EB
:105AB0009399090193D50501B3E5B90063FAA500EF
:105AC000B385250163E6250163F4A500B3852501AF
:105AD000B384A5406FF09FDFB7070001130A0001F0
:105AE000E36AF9F0130A80016FF0DFF0E3E8D5E82C
:105AF000B707010063FCF604930BF00F33B5DB002E
:105B00001315350033D7A60097A7010093870772B6
:105B1000B387E70083CB070093050002B38BAB008C
:105B2000338B7541631E0B0263E4360163EACC00DC
:105B30003384CC40B386D94033B58C00B384A640BF
:105B400013050400938504006FF05FE3B7070001BD
:105B500013050001E3E8F6FA130580016FF09FFAE0
:105B6000B3966601335D7601336DDD0033D4790180
:105B7000B395690133DC7C0193540D01336CBC0097
:105B80001305040093850400B31A6601EF00002199
:105B9000130A0500938504001305040033996C0172
:105BA000931C0D01EF00001B93DC0C011304050096
:105BB0009305050013850C00EF000017131A0A0166
:105BC00013570C013367EA00130A0400637EA70031
:105BD0003307A701130AF4FF6368A7016376A700E0
:105BE000130AE4FF3307A701B309A7409385040014
:105BF00013850900EF00801A938504001304050043
:105C000013850900EF0000159305050093040500B6
:105C100013850C00EF00401193150C0113140401BF
:105C200093D50501B365B4001387040063FEA50096
:105C3000B385A5011387F4FF63E8A50163F6A5000A
:105C40001387E4FFB385A501131A0A01B70C0100FD
:105C5000336AEA001384FCFFB3778A0033F48A00C6
:105C6000B384A54013850700930504002326F100A3
:105C7000135A0A01EF00400B930905009305040035
:105C800013050A00EF00400A13DC0A01930D05001A
:105C900093050C0013050A00EF0000098327C100DB
:105CA000130A050093050C0013850700EF00C007D9
:105CB0003305B50113D709013307A7006374B70192
:105CC000330A9A01B70701009387F7FF935507013D
:105CD0003377F70013170701B3F7F900B3854501D0
:105CE000B307F70063E6B400639EB400637CF90079
:105CF00033865741B3B7C700B385A541B385F54097
:105D000093070600B307F9403339F900B385B4406F
:105D1000B385254133947501B3D767013365F4002A
:105D2000B3D565016FF09FC513060500130500008C
:105D300093F61500638406003305C50093D515005E
:105D400013161600E39605FE678000006340050603
:105D500063C6050613860500930505001305F0FFCD
:105D6000630C060293061000637AB6006358C00005
:105D70001316160093961600E36AB6FE130500008C
:105D800063E6C500B385C5403365D50093D61600DC
:105D900013561600E39606FE67800000938200000B
:105DA000EFF05FFB13850500678002003305A0401C
:105DB00063D80500B305B0406FF0DFF9B305B0401C
:105DC00093820000EFF01FF93305A04067800200C6
:105DD0009382000063CA0500634C0500EFF09FF753
:105DE0001385050067800200B305B040E35805FE47
:105DF0003305A040EFF01FF63305B0406780020086
:02000004800278
:1000000049444C45000000006031FEFF2831FEFFEE
:100010003631FEFF4431FEFF4C31FEFF7032FEFFF1
:100020003832FEFF4632FEFF5432FEFF5C32FEFFE6
:10003000546D722053766300F437FEFFF437FEFFF1
:10004000F437FEFF7238FEFF4238FEFF6838FEFFCD
:10005000F437FEFFF437FEFF7238FEFF4238FEFF32
:10006000546D725100000000286E756C6C29000000
:10007000F645FEFFF447FEFFEA47FEFFF447FEFFAA
:10008000F447FEFFF447FEFFF447FEFF7446FEFF11
:10009000F447FEFFF447FEFF2C46FEFF8246FEFFBC
:1000A000F447FEFF3646FEFF4046FEFF4046FEFF99
:1000B0004046FEFF4046FEFF4046FEFF4046FEFF34
:1000C0004046FEFF4046FEFF4046FEFFF447FEFF6F
:1000D000F447FEFFF447FEFFF447FEFFF447FEFF40
:1000E000F447FEFFF447FEFFF447FEFFF447FEFF30
:1000F000F447FEFFF447FEFFF447FEFFF447FEFF20
:10010000F447FEFFF447FEFFF447FEFFF447FEFF0F
:10011000F447FEFFF447FEFFF447FEFFF447FEFFFF
:10012000F447FEFFF447FEFFF447FEFFF447FEFFEF
:10013000F447FEFFF447FEFFF447FEFFF447FEFFDF
:10014000F447FEFFF447FEFFF447FEFFF447FEFFCF
:10015000F447FEFFF447FEFFF447FEFFF447FEFFBF
:10016000F447FEFFF447FEFFF447FEFFF447FEFFAF
:10017000A646FEFF5247FEFFF447FEFFF447FEFF90
:10018000F447FEFFF447FEFFF447FEFFF447FEFF8F
:10019000F447FEFF9E46FEFFF447FEFFF447FEFFD6
:1001A000A647FEFFAC47FEFFF447FEFFF447FEFF05
:1001B000BA46FEFFF447FEFFA047FEFFF447FEFFEE
:1001C000F447FEFFC447FEFF6D69616F750A0000CA
:1001D0006D69616F75320A0068756E6772790A0021
:1001E0004572726F7220696E20416C74426C6F634D
:1001F0006B207461736B73200D0A000043686563A4
:100200006B54696D65720000416C74426C6F636B76
:100210005175657565000000464254657374310080
:100220004642546573743200000102020303030363
:100230000404040404040404050505050505050576
:100240000505050505050505060606060606060656
:10025000060606060606060606060606060606063E
:100260000606060606060606070707070707070726
:10027000070707070707070707070707070707070E
:1002800007070707070707070707070707070707FE
:1002900007070707070707070707070707070707EE
:1002A00007070707070707070808080808080808D6
:1002B00008080808080808080808080808080808BE
:1002C00008080808080808080808080808080808AE
:1002D000080808080808080808080808080808089E
:1002E000080808080808080808080808080808088E
:1002F000080808080808080808080808080808087E
:10030000080808080808080808080808080808086D
:10031000080808080808080808080808080808085D
:08032000080808080808080895
:100328001000000000000000017A5200017C010169
:100338001B0D02004C00000018000000084FFEFFD3
:10034800DC05000000440E307089039507810188A0
:100358000292049305940696089709980A990B9AAD
:100368000C0370020AC144C844C944D244D344D4DB
:1003780044D544D644D744D844D944DA440E00443A
:100388000B00000050000000680000009454FEFFBD
:100398000005000000440E507488028903930599F3
:1003A8000B810192049406950796089709980A9A72
:1003B8000C9B0D0320010AC144C844C944D244D34C
:1003C80044D444D544D644D744D844D944DA44DB49
:0803D800440E00440B0000007C
:1003EC00AAAAAAAA08000000FC8F010009000000BC
:040000058000004037
:00000001FF
